:100000000C94AA020C94EE020C94EE020C94EE02F4
:100010000C94EE020C94EE020C94EE020C94EE02A0
:100020000C94EE020C94EE020C94170D0C94E90D56
:100030000C94F51A0C94EE020C94EE020C94EE0261
:100040000C94EE020C94EE020C94EE020C94EE0270
:100050000C94EE020C945D1B0C94EE020C94EE02D8
:100060000C94EE020C94AF0F0C94EE020C94EE0282
:100070000C94EE020C94EE020C94EE020C94EE0240
:100080000C94EE020C94EE020C94EE020C94EE0230
:100090000C94EE020C94EE020C94EE020C94EE0220
:1000A0000C94EE020C94EE020C94EE02560E780EB6
:1000B000660F780E660FBD0EE00E660F350F480F07
:1000C00071127112A012A012DF12FF1255145514F2
:1000D0000A135514BA13BA1321142A1455144F14C1
:1000E000C713C713C713C713C713C713C713C71340
:1000F000C713C713C713C713C713C713C713C71330
:10010000D713E513EC13F313FD137500011E021E44
:10011000011F021F012002200121022101220222CF
:10012000012302230124022401250225012802289B
:10013000007500011E021E011F021F012002200186
:10014000210221012202220123022301240224018F
:1001500025022501280228007500011E021E011F2C
:10016000021F01200220012102210122022201237B
:100170000223012402240125022501280228002D42
:1001800021F1A1F1A2F1A33522E7323932E2A42B09
:1001900021000000C001C002C000000000000000FB
:1001A000000000000000000000000000000000004F
:1001B00000000000000000000000D200D000D129A3
:1001C0000014001A00090013000A000D000F0018A7
:1001D000001C00330034002A00C80004001500167B
:1001E00000170007000B00110008000C0012002887
:1001F000000000E1001D001B000600190005000EB4
:10020000001000360037003800C6000000C400E3CC
:1002100000C700C200C10000002C000000C500E6BD
:1002200000C300C00000000100CA00CB00CC0001E8
:100230000001000100010001000100010052004C1A
:1002400000010001000100010001000100010001A6
:10025000004A004B0050004F000000010001000167
:1002600000010001000100010001004D004E00519D
:100270000001000000010001000100010001000078
:100280000001000000010001000100010000000168
:10029000000100010001000100010001002400250F
:1002A00000260027000100010001000100010001FB
:1002B00000010001002F002100220023003700016F
:1002C00000000001000100010001000100010030F8
:1002D000001E001F0020003100010000000100DDB1
:1002E000000100010001000000480000002E002D68
:1002F0000001000100000001003A003B003C003D0D
:10030000003E003F004000410042004300440045E1
:1003100000010001000100010001000100010001D5
:1003200000010001000100010000000100010001C6
:1003300000010001000100010001000100010001B5
:1003400000010000000100010001000100010000A7
:100350000001000000010001000100010000000197
:10036000000100010001000100010001002400253E
:10037000002600270001000100010001000100012A
:1003800000010001002F002100220023003700019E
:100390000000000100010001000100010001003027
:1003A000001E001F0020003100010000000100DDE0
:1003B000000100010001000000480000002E002D97
:1003C000000100010000000A034A00440034003527
:1003D00000000012036700650065006B00680061A3
:1003E0000063006B000000040309040902740004A8
:1003F0000100A0FA09040000010301010009211114
:100400000100012240000705810308000A090401D8
:10041000000103010200092111010001224D000722
:1004200005820308000A0904020001030000000914
:1004300021110100012236000705830308000A0983
:100440000403000203000000092111010001222021
:1004500000070584032000010705040320000112A2
:1004600001100100000008EDFE60600100010200C3
:10047000010631FF0974A1010975150025FF9520BA
:10048000750881020976150025FF952075089102EF
:10049000C005010980A101850216010026B7001AD6
:1004A00001002AB700751095018100C0050C0901F3
:1004B000A1018503160100269C021A01002A9C0254
:1004C000751095018100C005010902A1010901A172
:1004D00000050919012905150025019505750181FA
:1004E0000295017503810105010930093115812546
:1004F0007F95027508810609381581257F9501755C
:10050000088106050C0A38021581257F95017508BA
:100510008106C0C005010906A101050719E029E708
:100520001500250195087501810295017508810165
:1005300005081901290595057501910295017503B5
:1005400091010507190029FF150026FF0095067582
:10055000088100C011241FBECFEFDAE0DEBFCDBF9F
:1005600004B603FE24C08091ED029091EE02A091AA
:10057000EF02B091F0028730904BA740B04BB9F436
:100580001092ED021092EE021092EF021092F00221
:1005900014BE84B7877F84BF88E10FB6F894809338
:1005A0006000109260000FBEE0E0F8E3099511E0F2
:1005B000A0E0B1E0EEEAF7E402C005900D92A434A9
:1005C000B107D9F712E0A4E4B1E001C01D92AD3E3D
:1005D000B107E1F70E94860A0C94D5230C94000021
:1005E00008950895279A2F988FEF9FEF9093870093
:1005F000809386008AE08093800089E18093810067
:100600000C94AC21282F81110BC080918000877F32
:100610008093800010928D0010928C002F98089586
:100620002F9880918000886080938000233019F497
:100630008FEF9FEF0FC083E090E0821B9109880F3E
:10064000991F2FEF3FEFA90102C0569547958A9554
:10065000E2F7CA0190938D0080938C0008950E9468
:10066000F2020C94F0020C94F102FC01613051F0A2
:1006700018F0623069F012C08281882379F088E531
:1006800091E008958281882349F081E391E0089503
:100690008281882319F08AE091E0089580E090E05B
:1006A000089581E0089581E008950C94530308951E
:1006B0000F931F93CF93DF938C01FC01C081D181F5
:1006C000CE010E94B919BE010E948906EC01B80151
:1006D0000E945503882309F470C1F80182818823A0
:1006E00009F45BC080914F0181111FC0C431F0E754
:1006F000DF0709F00AC10E94570381E080934F0190
:100700000E94271B90934E0180934D011092460149
:10071000109248011092470110924A01109249012B
:1007200010924C0110924B0148C180914D01909163
:100730004E010E94331B883C910570F48091460164
:10074000E82FF0E0EE0FFF1FE95BFE4FD183C0837F
:100750008F5F8093460131C1C43120E7D20708F092
:1007600024C1C23080E7D80710F5C11590E7D9073A
:1007700009F0DAC0F8018281882309F4BFC00E9421
:10078000C014FFEF24E38CE0F15020408040E1F7FB
:1007900000C000000E94821B10C1C431F0E7DF07D7
:1007A00008F0CFC0C23020E7D20708F49BC0F801A0
:1007B0008281882309F4A2C00E94341D811102C0E5
:1007C0000E94151D0E94511D90E09093DE028093BF
:1007D000DD02C230F0E7DF0721F48091DD028160A5
:1007E0007AC0C33020E7D20721F48091DD02826015
:1007F00072C0C43080E7D80721F48091DD028460A4
:100800006AC0C53090E7D90719F48091DD0227C08E
:10081000C630E0E7DE0721F48091DD0280615BC035
:10082000C730F0E7DF0721F48091DD02806253C01A
:10083000C83020E7D20721F48091DD0280644BC0EC
:10084000C93080E7D80721F48091DD02806843C079
:10085000CA3090E7D90729F48091DD02846088606E
:100860003AC0CB30E0E7DE0721F48091DD028E7FD5
:1008700032C0CC30F0E7DF0721F48091DD028D7FBC
:100880002AC0CD3020E7D20721F48091DD028B7F92
:1008900022C0CE3080E7D80719F48091DD021AC05B
:1008A0008091DD02CF3090E7D90711F48F7E13C01D
:1008B000C031E0E7DE0711F48F7D0DC0C131F0E7F4
:1008C000DF0711F48F7B07C0C231D04711F48F7757
:1008D00002C08B7F877F8093DD028091DD020E94C2
:1008E000551D6BC0C11580E7D80741F0C130D04716
:1008F000F1F081E08093440180934501C801DF91CC
:10090000CF911F910F910C945103C43120E7D2076E
:1009100008F04BC0C23080E7D80708F048CFC115B7
:1009200090E7D90709F42BCFC130D04711F7F80170
:100930008281882319F38091CC0281608093CC025C
:100940003CC0C333E0E7DE07A1F4F80182818823CD
:1009500021F01092440182E017C08091440181117E
:1009600006C086E20E94151186E20E94DD1182E037
:1009700019C0C433D04709F0BCCFF8018281882365
:1009800031F01092450180E20E942C1216C0809135
:100990004501811106C087E20E94151187E20E947D
:1009A000DD1180E20E94331208C0C333F0E7DF0795
:1009B00061F2C433D04709F39CCF80E0DF91CF913F
:1009C0001F910F9108950C942F030C9433032DE085
:1009D000729FF001112434E3839FE00DF11D112477
:1009E000E60FF11DEE0FFF1FE154FE4F859194912C
:1009F0000E949B06811540E5940708F047C08115C9
:100A000020E4920708F013C1883E910520F5803E4E
:100A1000910508F07CC1883A910578F4853A9105F2
:100A200008F0A5C08130910509F471C108F42EC108
:100A30008430910508F06BC129C18B3B910508F406
:100A4000A1C0803C910508F421C1FC01EE0FFF1FFD
:100A5000E150F040E6C0811530E2930758F481156B
:100A600041E0940708F053C1803F910508F40EC19E
:100A700090650895811520E3920708F0D5C0FC0128
:100A8000FF70EE0FFF1FE158FE4FCBC0811535E51B
:100A9000930708F043C0811544E5940708F0DEC0D1
:100AA000811522E5920708F5811531E5930708F0D5
:100AB000C1C0482F437021E030E002C0220F331F35
:100AC0004A95E2F73C68AC0164E0569547956A9513
:100AD000E1F74370342B8F708695869540E2849FB2
:100AE000C0011124822B932B0895282F269526953B
:100AF000AC01437055278115934508F0A0C080E2F2
:100B0000289F9001112481E090E002C0880F991F76
:100B10004A95E2F7822B932B9C6808958F3240E729
:100B2000940790F48F3120E7920708F0A2C0811556
:100B300036E5930708F497C09C01305621153041E3
:100B400008F0A4C09F7093C0803320E7920709F497
:100B500097C008F492C0813340E7940709F493C02A
:100B60008233904709F092C080E093ED0895853A72
:100B7000910509F48EC0863A910509F08DC082E88E
:100B800090E40895883A910509F489C0893A91055D
:100B900009F488C08A3A910509F487C08B3A910517
:100BA00009F486C08C3A910509F485C08D3A910507
:100BB00009F484C0803B910509F483C08E3A910505
:100BC00009F482C08F3A910509F481C0813B9105F7
:100BD00009F480C0823B910509F47FC0833B9105F5
:100BE00009F47EC0843B910509F47DC0853B9105E5
:100BF00009F47CC0863B910509F47BC0873B9105D5
:100C000009F47AC0883B910509F479C0893B9105C4
:100C100009F478C08A3B910509F477C080E094E438
:100C200008958591949108959927906C08959F70E7
:100C3000906A0895982F8827816F906A089590E2AE
:100C4000299F9001112481E090E002C0880F991F34
:100C50004A95E2F7822B932B9A680895982F88275C
:100C6000846F906A08958F719927982F88279062D2
:100C700008958F519047946D089580E091ED089507
:100C800080E090ED089580E092ED089580E090E09E
:100C9000089581E890E4089583E890E4089582EE51
:100CA00094E4089589EE94E408958AEE94E4089516
:100CB00085EB94E4089586EB94E4089587EB94E43F
:100CC00008958CEC94E408958DEC94E4089583E801
:100CD00095E408958AE895E4089582E995E40895F5
:100CE00084E995E4089581E296E4089583E296E428
:100CF000089584E296E4089585E296E4089586E2F4
:100D000096E4089587E296E408958AE296E40895C9
:100D100008959DE0799FF001112494E3899FE00DEF
:100D2000F11D1124E60FF11DEE0FFF1FE154FE4FE0
:100D30008591949108958238910549F1B0F48133F9
:100D4000910509F458C048F48932910509F44EC060
:100D50008A32910509F454C008958533910509F448
:100D600040C08933910599F00895833E910529F19A
:100D700038F4803E910591F0823E9105A1F00895EE
:100D8000863E9105F9F0873E910531F10895209155
:100D9000DD0220FD3AC021FD38C008958091DD02BA
:100DA00080FD35C032C08091DD0282FF32C080916B
:100DB000DD0284FD30C083EE39C08091DD0282FD0A
:100DC00028C0F5CF8091DD0283FF27C08091DD022E
:100DD00084FD21C087EE2AC08091DD0283FD1DC005
:100DE000F5CF8091DD0285FD1AC01BC08091DD0228
:100DF00085FD17C014C08091DD0286FD14C015C0AA
:100E00008091DD0286FD11C00EC080EE0FC089E327
:100E10000DC082EE0BC080E009C086EE07C089E2FB
:100E200005C085E303C08AE201C081E390E0089534
:100E300008950C941807E82FF0E0EF5DFE4F8081D5
:100E4000E82FEF70F0E082958F7021E030E0A9018B
:100E500002C0440F551F8A95E2F740A308950F93EF
:100E60001F93CF93DF9385B7806885BF85B7806870
:100E700085BFC3E0D0E001E010E0FE01EF5DFE4F72
:100E80008081E82FEF70F0E021A182958F70A8019A
:100E900002C0440F551F8A95E2F7CA01822B81A335
:100EA0008C2F0E941B07219740F78CE090E061E0B7
:100EB00070E0FC01EC5EFE4F2081E22FEF70F0E06D
:100EC00042A122952F70DB0102C0AA0FBB1F2A95F9
:100ED000E2F79D01242B22A3019758F7DF91CF91D0
:100EE0001F910F910C94E304EF92FF920F931F93C5
:100EF000CF93DF9308E511E0C3E0EE24E394F12CF7
:100F0000D5E08C2F0E941B078CE090E040E050E081
:100F1000FC01EC5EFE4F6081E62FEF70F0E020A157
:100F200030E062956F7002C0359527956A95E2F7BB
:100F300020FD09C09701082E02C0220F331F0A941A
:100F4000E2F7422B532B019718F7F8019291829107
:100F50008F018417950721F051834083D0930001BE
:100F60008C2F0E941B07C15060F68091000187FD05
:100F70002CC08150809300018F3F39F08FE99FE0B2
:100F80000197F1F700C0000020C0809156019091B8
:100F9000570190935F0180935E018091540190917D
:100FA000550190935D0180935C0180915201909175
:100FB000530190935B0180935A018091500190916D
:100FC000510190935901809358010E94E50481E0FA
:100FD000DF91CF911F910F91FF90EF900895E82F2F
:100FE000F0E0EE0FFF1FE85AFE4F808191810895D7
:100FF000089580916C0108950F931F93CF93DF9311
:1010000000D000D01F92CDB7DEB79C018091610166
:10101000909162012817390709F493C03093620157
:1010200020936101223E3105F1F1293E310559F14C
:101030002A3E310559F1253B310559F1263B310551
:1010400051F1273B310551F12C3C310561F12D3C2B
:10105000310531F1233881E0380729F12A3891E050
:10106000390709F1223981E03807E9F0243991E0A4
:101070003907C9F0213282E03807B9F0233292E013
:10108000390789F415C090E040E114C090E040E2D7
:1010900011C092E001C094E040E00CC090E1FCCFB0
:1010A00090E040E407C090E0F7CF90E044E002C059
:1010B00090E041E089018DEF4C839D830E94990F60
:1010C00080E00E94990F82E00E94990F4C81842F4A
:1010D0000E94990F9D81892F0E94990F80E00E94A4
:1010E000990F80E00E94990F80E00E94990F80E0A4
:1010F0000E94990F8091E302843019F583E089837F
:101100001B830A838093E9008FEF9091E800815060
:1011100095FD06C095ED9A95F1F700008111F5CF88
:101120008091E80085FF0DC040E050E063E070E092
:10113000CE0101960E94070B8091E8008E77809384
:10114000E8000F900F900F900F900F90DF91CF91CC
:101150001F910F910895CF93DF9300D01F92CDB7C9
:10116000DEB72091E302243021F522E029839B831E
:101170008A8383E08093E9008FEF9091E8008150AB
:1011800095FD06C095ED9A95F1F700008111F5CF18
:101190008091E80085FF0DC040E050E063E070E022
:1011A000CE0101960E94070B8091E8008E77809314
:1011B000E8000F900F900F90DF91CF910895CF939B
:1011C000DF93EC018DEF0E94990F80E00E94990F50
:1011D00083E00E94990F88810E94990F89810E9463
:1011E000990F8A810E94990F8B810E94990F8C819F
:1011F0000E94990F80E00E94990F8091E302843051
:10120000F9F482E08093E9008FEF9091E80081503B
:1012100095FD06C095ED9A95F1F700008111F5CF87
:101220008091E80085FF0CC040E050E065E070E090
:10123000CE010E94070B8091E8008E778093E80032
:10124000DF91CF910895EF92FF920F931F93CF9369
:10125000DF93EC018DEF0E94990F8E017E0188E0F3
:10126000E80EF11CF80181918F010E94990F0E1573
:101270001F05C1F78091E302843039F581E0809346
:10128000E9008FEF9091E800815095FD06C0F5EDE3
:10129000FA95F1F700008111F5CF8091E80085FF04
:1012A00014C040E050E068E070E0CE010E94070BFF
:1012B0008091E8008E778093E80088E0FE01A4E644
:1012C000B1E001900D928A95E1F7DF91CF911F91E6
:1012D0000F91FF90EF9008958091E202811109C073
:1012E0000E949C0C0E94F90C8091E2008460809323
:1012F000E20008951092E2020895089508950C9472
:10130000EA1A209160012F5F822F62E30E94652319
:10131000992319F020936001089510926001809143
:101320006301882371F18091E302843041F580915B
:10133000E9008F702091EC00922F917020FD90E8D1
:10134000892B94E09093E9009091EB0090FF14C0FA
:101350009091EE0097FF10C09091E80095FF03C0B8
:101360001092F100F9CF9091E80090FF05C09091A4
:10137000E8009E779093E8008F708093E9001092C8
:101380006301089542E061EC81E00E94160C42E0A6
:1013900061EC82E00E94160C42E061EC83E00E9466
:1013A000160C42E261EC84E00C94160C8091E5028C
:1013B000833009F453C030F4813071F0823009F485
:1013C0008CC008958A3009F478C08B3009F45EC06F
:1013D000893009F09AC020C08091E402813A09F076
:1013E00094C08091E800877F8093E8008091E802B4
:1013F0009091E902892B21F468E084E691E003C032
:1014000060E080E090E070E00E94520B8091E80084
:101410008B778093E80008958091E402813209F08F
:1014200074C08091E8029091E902892B09F06DC0A7
:101430008091E800877F8093E8008091E80082FD3A
:1014400005C08091E3028111F8CF5FC08091F10067
:1014500080936C018091E8008B7753C08091E40207
:10146000813A09F052C08091E8029091E902892BFB
:1014700009F04BC08091E800877F8093E80080915D
:10148000E80080FFFCCF80910B0136C08091E40220
:101490008132D9F58091E8029091E902892BA9F572
:1014A0008091E800877F8093E8000E944B0C809138
:1014B000E60280930B010C94C0148091E402813207
:1014C00021F58091E800877F8093E8000E944B0C13
:1014D0008091E70280936D0108958091E402813A42
:1014E000A1F48091E800877F8093E8008091E80074
:1014F00080FFFCCF80916D018093F1008091E80026
:101500008E778093E8000C944B0C089584B7877F06
:1015100084BF88E10FB6F894809360001092600059
:101520000FBE80E880936100109261000E942D1030
:101530000E949C0C0E94F90C8091E20084608093D0
:10154000E20078940E949B0F0E947E0F0E942F1051
:1015500081E091E00E94D90F0E943710FDCF292F22
:10156000332723303105C9F064F42130310581F08F
:101570002230310509F043C084E790E02BEE33E0E0
:1015800042C021323105F1F02232310541F137C03C
:1015900082E190E02FE534E036C099278130910553
:1015A00041F08230910541F0892B49F5E7EEF3E0F7
:1015B00005C0E3EDF3E002C0E7ECF3E0849190E0D6
:1015C0009F0121C06430D8F4E62FF0E0EE0FFF1F3A
:1015D000EF5CFE4F2081318189E090E014C06430DF
:1015E00070F470E0FB01EE0FFF1FE75DFE4F2081FE
:1015F0003181FB01EB5DFE4F808190E004C080E013
:1016000090E020E030E0FA01318320830895CF920A
:10161000DF92EF92FF920F931F93CF93DF93EC0132
:101620008B016A010E946A0C811133C0C114D1047C
:1016300039F0F60180819181081B190BC80FD91F61
:10164000E12CF12C0115110519F18091E80085FDBF
:1016500016C08091E8008E778093E800C114D10411
:1016600049F0F60180819181E80EF91EF182E08255
:1016700085E00FC00E946A0C882321F30AC089917B
:101680008093F10001501109FFEFEF1AFF0ADACF42
:1016900080E0DF91CF911F910F91FF90EF90DF904D
:1016A000CF9008952091EA023091EB022617370778
:1016B00048F06115710539F42091E8002E772093E8
:1016C000E80001C0B90140E061157105A9F1209160
:1016D000E302222309F443C0253009F442C02091DB
:1016E000E80023FD40C02091E80022FD32C0209197
:1016F000E80020FFE9CF4091F3002091F20030E0B4
:10170000342BFC01CF016115710559F028303105EA
:1017100040F481918093F100615071092F5F3F4F38
:10172000F1CF41E02830310509F040E02091E80098
:101730002E772093E800C8CF4111C9CF0AC080910D
:10174000E302882361F0853061F08091E80083FD39
:101750000AC08091E80082FFF2CF80E0089582E025
:10176000089583E0089581E008952091EA02309180
:10177000EB022617370748F06115710539F42091FF
:10178000E8002E772093E80001C0B901FC0120E0B9
:101790006115710591F18091E302882309F440C03D
:1017A000853009F43FC08091E80083FD3DC0809101
:1017B000E80082FD2FC08091E80080FFE9CF2091F2
:1017C000F3008091F20090E0922B6115710559F0C1
:1017D0008830910540F424912093F10031966150B6
:1017E00071090196F2CF21E0089709F020E080917D
:1017F000E8008E778093E800CBCF2111CCCF0AC0D0
:101800008091E302882361F0853061F08091E800E7
:1018100083FD0AC08091E80082FFF2CF80E0089546
:1018200082E0089583E0089581E00895982F97302D
:1018300058F59093E900981739F07091EC002091D9
:10184000ED005091F00003C0242F762F50E021FFCF
:1018500019C03091EB003E7F3093EB003091ED00EA
:101860003D7F3093ED003091EB0031603093EB0021
:101870007093EC002093ED005093F0002091EE0067
:1018800027FF07C09F5FD3CF8F708093E90081E06F
:10189000089580E008958091E40287FF11C080914F
:1018A000E80082FD05C08091E3028111F8CF11C0EC
:1018B0008091E8008B770BC08091E302882349F088
:1018C0008091E80080FFF8CF8091E8008E778093C8
:1018D000E80008952091E4003091E50095E64091FC
:1018E000EC00842F817040FF22C08091E80080FDD1
:1018F0001CC08091E302882391F0853091F08091A3
:10190000EB0085FD10C04091E4005091E5004217C6
:10191000530729F39A01915011F784E0089582E06A
:10192000089583E0089581E0089580E0089540914E
:10193000E80042FFDECF08950E940A0D0E94120DBA
:10194000E0EEF0E0808181608083E8EDF0E080816E
:101950008F77808319BCA7EDB0E08C918E7F8C933C
:1019600080818F7E80831092E20208950F931F93EF
:10197000CF93DF930E940A0D0E94120DC8EDD0E0B4
:1019800088818F77888388818068888388818F7D2C
:10199000888319BC1092E3021092DF021092E102D8
:1019A0001092E00200EE10E0F80180818B7F8083CE
:1019B00088818160888342E060E080E00E94160CAC
:1019C000E1EEF0E080818E7F8083E2EEF0E08081C6
:1019D00081608083808188608083F80180818E7F30
:1019E0008083888180618883DF91CF911F910F91DF
:1019F0000895E8EDF0E080818F7E8083E7EDF0E0F0
:101A000080818160808384E082BF81E08093E202F4
:101A10000C94B60CE8EDF0E080818E7F808310920C
:101A2000E20008951092DA001092E10008951F92EA
:101A30000F920FB60F9211242F933F934F935F9302
:101A40006F937F938F939F93AF93BF93EF93FF9386
:101A50008091E10082FF0BC08091E20082FF07C00D
:101A60008091E1008B7F8093E1000E948109809149
:101A7000DA0080FF1FC08091D80080FF1BC08091DA
:101A8000DA008E7F8093DA008091D90080FF0DC04C
:101A900080E189BD82E189BD09B400FEFDCF81E00E
:101AA0008093E3020E946C0905C019BC1092E30206
:101AB0000E947A098091E10080FF19C08091E200C4
:101AC00080FF15C08091E2008E7F8093E2008091BC
:101AD000E20080618093E2008091D8008062809370
:101AE000D80019BC85E08093E3020E947E098091B2
:101AF000E10084FF30C08091E20084FF2CC080E1CF
:101B000089BD82E189BD09B400FEFDCF8091D80076
:101B10008F7D8093D8008091E1008F7E8093E100DB
:101B20008091E2008F7E8093E2008091E2008160EC
:101B30008093E2008091DF02882311F084E007C0E7
:101B40008091E30087FD02C081E001C083E08093C3
:101B5000E3020E947F098091E10083FF29C0809108
:101B6000E20083FF25C08091E100877F8093E10040
:101B700082E08093E3021092DF028091E1008E7F89
:101B80008093E1008091E2008E7F8093E20080915B
:101B9000E20080618093E20042E060E080E00E9429
:101BA000160C8091F00088608093F0000E947D09FF
:101BB000FF91EF91BF91AF919F918F917F916F9125
:101BC0005F914F913F912F910F900FBE0F901F90FB
:101BD00018951F920F920FB60F9211242F933F93D7
:101BE0004F935F936F937F938F939F93AF93BF9325
:101BF000CF93DF93EF93FF93C091E900CF70809173
:101C0000EC00D82FD17080FDD0E81092E9008091CF
:101C1000F000877F8093F00078940E942D0E109240
:101C2000E9008091F00088608093F000CD2BCF70A8
:101C3000C093E900FF91EF91DF91CF91BF91AF91F8
:101C40009F918F917F916F915F914F913F912F91D4
:101C50000F900FBE0F901F9018951F93CF93DF9397
:101C6000CDB7DEB7AA970FB6F894DEBF0FBECDBFD3
:101C7000E4EEF2E088E08E0F9091F10091938E13E4
:101C8000FBCF0E94D6098091E80083FF1FC180919D
:101C9000E4029091E502492F50E04A30510508F0E6
:101CA00015C1FA01EA5AFF4F0C948523803881F060
:101CB000823809F00BC18091E8028F708093E900AF
:101CC0008091EB0085FB882780F91092E90006C01F
:101CD0008091E0029091E102911182609091E80080
:101CE000977F9093E8008093F1001092F100C8C0B4
:101CF000282F2D7F09F0EAC0882319F0823061F087
:101D0000E5C08091E602813009F0E0C0933009F02F
:101D100080E08093E1022BC08091E602811127C010
:101D20008091E8028F7009F4D1C08093E90020917E
:101D3000EB0020FF1CC0933021F48091EB00806207
:101D400014C09091EB0090619093EB0021E030E0A3
:101D5000A90102C0440F551F8A95E2F74093EA009B
:101D60001092EA008091EB0088608093EB00109263
:101D7000E9008091E800877F86C08111A7C010919B
:101D8000E6021F778091E3008078812B8093E30047
:101D90008091E800877F8093E8000E944B0C80913F
:101DA000E80080FFFCCF8091E30080688093E3002F
:101DB000111102C082E001C083E08093E30286C07B
:101DC0008058823008F082C08091E6029091E7024C
:101DD0008C3D53E0950779F583E08A838AE2898315
:101DE0004FB7F894DE01139620E03EE051E2E32F76
:101DF000F0E050935700E49120FF03C0E295EF70AC
:101E00003F5FEF708E2F90E0EA3010F0C79601C070
:101E1000C0968D939D932F5F243149F74FBF8091DA
:101E2000E800877F8093E8006AE270E0CE010196C7
:101E30000E94520B14C0AE014F5F5F4F6091E802E9
:101E40000E94AF0ABC01009709F440C09091E800DD
:101E5000977F9093E80089819A810E94B50B8091C9
:101E6000E8008B778093E80031C0803879F5809165
:101E7000E800877F8093E8008091DF028093F10083
:101E80008091E8008E778093E8000E944B0C1EC082
:101E900081111CC09091E6029230C0F48091E8005C
:101EA000877F8093E8009093DF020E944B0C809123
:101EB000DF02811106C08091E30087FD02C081E04E
:101EC00001C084E08093E3020E94C2098091E8008F
:101ED00083FF0AC08091E800877F8093E8008091AB
:101EE000EB0080628093EB00AA960FB6F894DEBFF9
:101EF0000FBECDBFDF91CF911F910895CF938091F9
:101F0000E3028823A1F0C091E900CF709091EC002A
:101F1000892F817090FD80E8C82B1092E900809194
:101F2000E80083FD0E942D0ECF70C093E900CF9191
:101F300008950C94A80F87E68093CC001092CD00F2
:101F400088E08093C90086E08093CA007894089561
:101F50009091C80095FFFCCF8093CE0008951F920A
:101F60000F920FB60F9211242F933F934F938F939D
:101F70009F93EF93FF9380916F0190E09C012F5FFF
:101F80003F4F40916E01421741F03091CE00FC016D
:101F9000E059FE4F308320936F01FF91EF919F91A5
:101FA0008F914F913F912F910F900FBE0F901F90E7
:101FB000189590937502809374020895E0917402CD
:101FC000F0917502309721F00190F081E02D099495
:101FD00080E00895E0917402F0917502309721F04D
:101FE0000280F381E02D09940895E0917402F0914C
:101FF0007502309721F00480F581E02D0994089551
:1020000020917202309173028217930771F09093BE
:10201000730280937202E0917402F091750230971E
:1020200021F00680F781E02D099408952091700237
:10203000309171028217930771F09093710280932F
:102040007002E0917402F0917502309721F00084E3
:10205000F185E02D0994089508950C942C100E94A8
:102060001E1B0E942F070E94EC1B0C94AC215F9258
:102070006F927F928F929F92AF92BF92CF92DF9298
:10208000EF92FF920F931F93CF93DF9300D000D076
:102090001F92CDB7DEB70E9474079FE7C92E92E06A
:1020A000D92E03E010E0AA24A394B12C502E802F47
:1020B0000E94EF074C01F601729062906F01682652
:1020C000792661147104A1F40150110978F78FEF9A
:1020D00089838A831B820E94271B8160782F9D83BE
:1020E0008C8349815A816B818D810E94E71038C0B1
:1020F0008091CC0281FD0E94F8072CE030E0750150
:10210000022E02C0EE0CFF1C0A94E2F7C7018621E2
:102110009721892B09F129835A828E209F2091E0F3
:10212000892809F490E09B830E94271B8160782F07
:102130009D838C8349815A816B818D810E94E71038
:10214000000F111FF801E958FD4F80819181E826A9
:10215000F926F182E08204C02150310980F6B4CF23
:102160000E94DD1E109176020E94DE0F1817D1F03A
:102170000E94DE0F809376020F900F900F900F90C9
:102180000F90DF91CF911F910F91FF90EF90DF9013
:10219000CF90BF90AF909F908F907F906F905F9007
:1021A0000C9419070F900F900F900F900F90DF91E4
:1021B000CF911F910F91FF90EF90DF90CF90BF9044
:1021C000AF909F908F907F906F905F900895CF9386
:1021D000DF93CDB7DEB72B970FB6F894DEBF0FBEF7
:1021E000CDBF4F83588769877A878B87DE01119629
:1021F00086E0FD0111928A95E9F785E0FE013796A8
:1022000001900D928A95E1F749815A816B817C8119
:102210008D819E810E945E172B960FB6F894DEBFCB
:102220000FBECDBFDF91CF910895CF93882309F4DE
:10223000C2C0C82F823859F40E94DE0F81FDBBC096
:1022400089E30E94381A0E94BB1A89E30CC08338C4
:1022500079F40E94DE0F80FDAEC083E50E94381A3B
:102260000E94BB1A83E50E94551ACF910C94BB1AA9
:10227000843859F40E94DE0F82FD9DC087E40E94DD
:10228000381A0E94BB1A87E4EECF8CEF8C0F813A8C
:1022900048F48C2F0E94152181118DC08C2F0E9433
:1022A000381AE3CF80E28C0F883048F4C77081E0A1
:1022B00001C0880FCA95EAF70E94741AD6CF8BE541
:1022C0008C0F833078F4C53A29F0C63A31F083E8B0
:1022D00090E005C081E890E002C082E890E0CF91F4
:1022E0000C94001088E58C0F833108F064C0C83A64
:1022F00039F1C93A41F1CA3A49F1CB3A51F1CC3AF4
:1023000059F1CD3A61F1C03B69F1CE3A71F1CF3A62
:1023100079F1C13B81F1C23B89F1C33B91F1C43BEF
:1023200099F1C53BA1F1C63BA9F1C73BB1F1C83B4F
:10233000B9F1C93BC1F1CA3BC9F180E090E038C0B6
:1023400082EE90E035C089EE90E032C08AEE90E0F7
:102350002FC085EB90E02CC086EB90E029C087EB86
:1023600090E026C08CEC90E023C08DEC90E020C083
:1023700083E891E01DC08AE891E01AC082E991E00B
:1023800017C084E991E014C081E292E011C083E2B9
:1023900092E00EC084E292E00BC085E292E008C0B9
:1023A00086E292E005C087E292E002C08AE292E013
:1023B000CF910C941610CF910895882309F44BC047
:1023C000823859F40E94DE0F81FF45C089E30E94E4
:1023D000381A0E94BB1A89E30CC0833871F40E943A
:1023E000DE0F80FF38C083E50E94381A0E94BB1AB6
:1023F00083E50E94551A0C94BB1A843859F40E9444
:10240000DE0F82FF28C087E40E94381A0E94BB1AA0
:1024100087E4EFCF9CEF980F913A58F390E2980F32
:10242000983050F4877091E001C0990F8A95EAF7CF
:10243000892F0E947A1ADFCF9BE5980F933020F402
:1024400080E090E00C940010885A833120F480E002
:1024500090E00C9416100895882321F00E94741ABD
:102460000C94BB1A0895882321F00E947A1A0C94C8
:10247000BB1A08957F928F929F92AF92BF92CF9294
:10248000DF92EF92FF920F931F93CF93DF931F92F0
:10249000CDB7DEB77C01C62E772EFC0105810295F3
:1024A0000F70128111110E94911A0E94311A882313
:1024B00079F0112369F080E28C0D883048F082E0D9
:1024C0000E941A1A0E94311A91E0D82ED92601C012
:1024D000D12CE72DE295EF70F0E0E05AFF4F0C941D
:1024E0008523872D807F072D0F70882311F002959B
:1024F000007F112389F0002309F499C180E28C0D3B
:10250000883020F4802F0E94741A03C0802F0E940C
:10251000841A0E94BB1A8BC18C2D0E94DD110023EE
:1025200009F4C3C180E28C0D883020F4802F0E9412
:102530007A1A03C0802F0E948A1A0E94BB1AB5C162
:10254000872D807F972D9F70803211F4892F03C0D3
:10255000892F8295807FCC2021F0F1E0CF16A1F069
:102560001DC0112339F0002319F1013009F50E9433
:10257000A41A9BC1002319F0013009F496C1898384
:102580000E94A71A898110C1112321F0063008F09A
:102590008CC10EC0053008F088C106C1112359F066
:1025A000002331F0F701958190FF41C19F70958321
:1025B0000E942C127AC1002309F4F6C03EC1872D77
:1025C00086958695837090E0009719F0019761F0E9
:1025D0006CC1112321F08C2D972D937002C080E0E7
:1025E00090E00E94001061C1112321F08C2D972DE5
:1025F000937002C080E090E00E94161056C18C2DAE
:10260000112319F00E94E51D02C00E944D1E0E9478
:10261000D21E4BC1872D837009F052C0111145C1E4
:102620008C2D829586958770880F880F9C2D9F70C2
:10263000892E912CA12CB12C082E04C0880C991C39
:10264000AA1CBB1C0A94D2F7C4FE14C00FE010E011
:1026500020E030E0B901A80104C0440F551F661FF7
:10266000771F8A95D2F7CB01BA0160957095809556
:10267000909503C060E070E0CB01272D269526954C
:10268000237030E02230310569F02330310589F0C4
:10269000682979298A299B292130310571F00E9406
:1026A000A61803C1682979298A299B290E94C21882
:1026B000FCC00E94A618C501B4010E948A18F5C08A
:1026C000112319F0872D817001C08695882309F4A4
:1026D000ECC08C2D829586958770880F880F9C2D75
:1026E0009F70892E912CA12CB12C082E04C0880C2F
:1026F000991CAA1CBB1C0A94D2F7C4FE14C00FE09C
:1027000010E020E030E0B901A80104C0440F551FDB
:10271000661F771F8A95D2F7CB01BA016095709535
:102720008095909503C060E070E0CB01272D269541
:1027300026952370422F50E04230510569F0433016
:10274000510589F0682979298A299B294130510549
:1027500071F00E948019A9C0682979298A299B29CA
:102760000E949C19A2C00E948019C501B4010E9458
:1027700064199BC08C2D90E0FC01E05EF109E5310D
:10278000F10508F050C0E059FF4F0C9485230C2D43
:102790000F70872D8F71112321F00E94FD18802F5B
:1027A00007CF0E941E19802F0E9433127EC0112372
:1027B00041F0053008F079C0872D8F710E944319D0
:1027C00074C0063008F071C0F7CF112339F0872D9F
:1027D0008F710E94FD1869C01123C9F3872D8F7175
:1027E0000E941E1962C0112329F0872D8F710E944B
:1027F000E8185BC00E94DE1858C0112351F0172D55
:102800001F71812F0E94FD1863E0812F0E94111A11
:102810004CC081E00E941A1A023008F446C082E0DF
:102820000E941A1A42C0112331F0002381F28C2D2C
:102830000E9415113AC0002389F28C2D0E94DD11EF
:1028400034C0472D4F706C2DC7010E9435030E9484
:1028500002182BC0111129C0472D4F7050E0423093
:102860005105B9F04CF44115510581F04130510545
:10287000E1F40E94D42119C04330510569F044307D
:10288000510599F48C2D0E9426220FC00E94BD2173
:102890000CC00E94F02109C00E94032206C0472DEF
:1028A0004F706C2DC7010E948806DD20F9F00E9450
:1028B0000D1A80FD1BC0F70112820E94071A0E94A8
:1028C000FD18C7010E9485140E94071A0F90DF911E
:1028D000CF911F910F91FF90EF90DF90CF90BF901D
:1028E000AF909F908F907F900C941E190F90DF9166
:1028F000CF911F910F91FF90EF90DF90CF90BF90FD
:10290000AF909F908F907F9008950F931F93CF93D8
:10291000DF93EC01888199812B813C81232BB9F0D5
:102920009F3F11F48F3F99F0CE010E9458038823F6
:1029300071F0688179818A810E94031A8C010E945A
:10294000B8190E947F18B801CE010E943A12DF9197
:10295000CF911F910F9108950E94911A0E94A11A80
:102960000E94661A0E94BB1A0E94831F0E94D21EF8
:1029700080E090E00E94001080E090E00C9416103F
:102980000E94811A0C94AC140E94F819292F2295E8
:102990002F7030E02C3031054CF42A3031056CF4C6
:1029A0002250310922303105A8F407C02C303105FE
:1029B00069F02F30310551F00DC0803F69F018F4F7
:1029C000803E40F409C0843F29F406C093FB882769
:1029D00080F9089580E0089581E00895CF93DF9312
:1029E00000D000D01F92CDB7DEB70F900F900F90A0
:1029F0000F900F90DF91CF910895CF93DF9300D088
:102A000000D000D0CDB7DEB726960FB6F894DEBF63
:102A10000FBECDBFDF91CF9108951F93CF93DF936A
:102A2000C0917F0216E080918002C81799F0D0E033
:102A30001C9FF0011D9FF00D1124EF57FD4F4081A9
:102A4000518162817381848195810E94FD14219658
:102A5000C770E9CFDF91CF911F9108954091B102E6
:102A60005091B2026091B3027091B4028091B502AC
:102A70009091B6020C94FD148091B60282958F70ED
:102A800009F054C08091B302882309F44FC08091AB
:102A90007F02A09180026091B1027091B2024091D8
:102AA000B4025091B502B6E08A1709F43FC090E035
:102AB00041155105C1F17F3F11F46F3FA1F1B89F5E
:102AC000F001B99FF00D1124EF57FD4F21817213D2
:102AD0002AC02081621327C02281211124C02381B2
:102AE00034812417350710F421503109241B350B8C
:102AF000283C3105C0F42091B6022F70206120934C
:102B0000B60226E0289FF001299FF00D1124EA5714
:102B1000FD4F80818F708061808381EB92E00E9405
:102B200085140C940D1501968770BECF0895CF9231
:102B3000DF92EF92FF920F931F93CF93DF93CDB766
:102B4000DEB762970FB6F894DEBF0FBECDBF8C0123
:102B500085E0F801DE011D9601900D928A95E1F75E
:102B6000D8014C9111965C91119712966C91129725
:102B70001396CD90DC9014973091B1027091B2020F
:102B80008091B4029091B502009709F46BC17F3F28
:102B900019F43F3F09F466C1E090B302EE2009F456
:102BA000C0C02091B602C816D90628F0F601E81B6D
:102BB000F90BCF0104C0809590958C0D9D1DFF24CD
:102BC000F394883C910578F0F12C207F09F0C6C081
:102BD0007C2DD98AC88A89890E94EE1481EB92E003
:102BE0000E948514B1C0822F807F09F046C0751302
:102BF00014C0341312C0611110C02F7020612093D3
:102C0000B6020E942E1581EB92E00E9485148091FD
:102C1000B602D80115968C932EC0CD2819F15F3FCE
:102C200011F44F3FF9F0F62E61111CC080917F0224
:102C30002091800236E0821709F45AC090E0389F54
:102C4000F001399FF00D1124EF57FD4F718157139B
:102C500006C07081471303C07281711103C00196D1
:102C60008770E9CFF62E662309F418C18091B60269
:102C700081608093B602F12C11C1751308C0341322
:102C800006C0611104C08091B602D801C3C04D874F
:102C90005E878D859E856A8B0E94C4146A8988230D
:102CA000E1F16623D1F12091B602822F82958F70D7
:102CB00090E0029774F08091B1029091B2029887EF
:102CC0008F831986DB86CA862C87CE0107960E94E1
:102CD000851486E0F801A1EBB2E001900D928A958F
:102CE000E1F70E943C150E942E15FF24F394D6C0F4
:102CF0004D875E878D859E850E94F819292F229524
:102D00002F7030E0223031050CF0BCC09F7009F00C
:102D1000B6C0805E883008F4C1C0C8010E94851426
:102D2000E4CFC816D90608F453C0F601E81BF90B26
:102D3000CF01883C910508F450C0F12C7C2DD98A34
:102D4000C88A89890E94EE14E1EBF2E086E0DF0197
:102D50001D928A95E9F70E942E15A0C0751314C024
:102D6000341312C0611110C08091B602F80185833E
:102D7000C8010E94851486E0E1EBF2E0DF011D92BC
:102D80008A95E9F7FE2C8AC04D875E878D859E85E2
:102D90006A8B0E94C4146A89882309F4BECF662313
:102DA00009F4BBCF2091B602822F82958F7090E0FC
:102DB00002970CF48ECF8091B1029091B2029A8367
:102DC00089831B82DD82CC822E83CE0101967FCF48
:102DD000809590958C0D9D1DACCFF62E662309F441
:102DE0009CCF75132EC034132CC02091B60220FD49
:102DF0001FC0822F82958F70D9F0D80115962C9321
:102E000015978F3049F08F5F982F9295907F822F82
:102E10008F70892B15968C93C8010E94851486E0CB
:102E2000F801A1EBB2E001900D928A95E1F793CF02
:102E300086E0F801A1EBB2E001900D928A95E1F7EE
:102E40002DC04D875E878D859E850E94C41481119B
:102E500040CF8091B60281608093B602C8010E9483
:102E600085141CC0662309F458CF4D875E878D8575
:102E70009E850E94C414882309F44FCF2ACF811164
:102E800048CF0CC0243031050CF047CF9F7009F4B7
:102E900040CFF8019581907F09F03BCF8F2D62964E
:102EA0000FB6F894DEBF0FBECDBFDF91CF911F915B
:102EB0000F91FF90EF90DF90CF9008951F93CF93E5
:102EC000DF93CDB7DEB72C970FB6F894DEBF0FBEF9
:102ED000CDBF4F83588769877A878B879C87CE01C0
:102EE00007960E949715882369F08F8198852A8517
:102EF0003B85232BF1F19F3F09F063C08F3F09F021
:102F000060C037C086E0FE013796DE011196019061
:102F10000D928A95E1F76F817885EA85FB85309778
:102F200041F17F3F11F46F3F21F12091800230E0A9
:102F3000C90101968770992740917F0250E084175C
:102F4000950709F447C069837A83FD83EC8396E093
:102F5000929FD001939FB00D1124AF57BD4FFE013A
:102F6000319601900D929A95E1F7809380020E942C
:102F70000D1516E080917F02909180028917C1F1B2
:102F8000189FC00111248F579D4F0E9497158823C9
:102F900079F1E0917F021E9FF0011124EF57FD4F60
:102FA0004081518162817381848195810E94FD14E9
:102FB00080917F0290E001968770992780937F022D
:102FC000D9CF4F81588569857A858B859C850E94EC
:102FD000FD14CFCF0E94C0141092800210927F0285
:102FE000E1EBF2E086E0DF011D928A95E9F7C1CFBF
:102FF0002C960FB6F894DEBF0FBECDBFDF91CF91F8
:103000001F910895EF92FF920F931F93CF93DF9339
:103010008C01009709F46CC0F12CEE24E394E801D4
:103020002196F8018491843740F4843008F051C02F
:10303000813081F0823019F15BC0853709F444C0DA
:10304000A8F19CE7980F903708F052C08F770E9444
:10305000DD1141C00E5F1F4FFE01C49180E28C0F55
:10306000883048F4C7708E2D01C0880FCA95EAF7E2
:103070000E94941A14C08C2F0E9415112DC00E5F4F
:103080001F4FFE01C49180E28C0F883058F4C77046
:103090008E2D01C0880FCA95EAF70E949A1A0E94E5
:1030A000BB1A1AC08C2F0E94DD1116C00E5F1F4F75
:1030B000FE01C491CC2381F08FE99FE00197F1F7E5
:1030C00000C00000C150F6CF0E5F1F4FFE01F4900C
:1030D00003C00E9415118E018F2D882309F49FCF04
:1030E000EFE9FFE03197F1F700C000008150F5CF24
:1030F000DF91CF911F910F91FF90EF900895089568
:103100006093BB027093BC028093BD029093BE0299
:103110000C94AC140F931F930091BB021091BC024E
:103120002091BD023091BE02DC01CB01802B912B9E
:10313000A22BB32B8093BB029093BC02A093BD0241
:10314000B093BE021F910F910C94AC140F931F9378
:103150000091BB021091BC022091BD023091BE02D1
:10316000DC01CB0180239123A223B3238093BB02F4
:103170009093BC02A093BD02B093BE021F910F9129
:103180000C94AC140F931F930091BB021091BC02DE
:103190002091BD023091BE02DC01CB018027912736
:1031A000A227B3278093BB029093BC02A093BD02D9
:1031B000B093BE021F910F910C94AC141092B70201
:1031C0001092B8021092B9021092BA020C94AC1488
:1031D00041E050E060E070E004C0440F551F661FFE
:1031E000771F8A95D2F74093B7025093B802609345
:1031F000B9027093BA020C94AC1441E050E060E064
:1032000070E004C0440F551F661F771F8A95D2F7E0
:103210008091B7029091B802A091B902B091BA0220
:10322000482B592B6A2B7B2B4093B7025093B80243
:103230006093B9027093BA020C94AC1441E050E070
:1032400060E070E004C0440F551F661F771F8A9529
:10325000D2F740955095609570958091B702909106
:10326000B802A091B902B091BA02482359236A2347
:103270007B234093B7025093B8026093B9027093D6
:10328000BA020C94AC1441E050E060E070E004C07D
:10329000440F551F661F771F8A95D2F78091B7029A
:1032A0009091B802A091B902B091BA02482759276B
:1032B0006A277B274093B7025093B8026093B90204
:1032C0007093BA020C94AC140F931F930091B70241
:1032D0001091B8022091B9023091BA02DC01CB0101
:1032E000802B912BA22BB32B8093B7029093B80223
:1032F000A093B902B093BA021F910F910C94AC1431
:103300000F931F930091B7021091B8022091B90258
:103310003091BA02DC01CB0180239123A223B32395
:103320008093B7029093B802A093B902B093BA0207
:103330001F910F910C94AC140F931F930091B7023F
:103340001091B8022091B9023091BA02DC01CB0190
:1033500080279127A227B3278093B7029093B802C2
:10336000A093B902B093BA021F910F910C94AC14C0
:103370000895CF92DF92EF92FF920F931F93CF9316
:10338000DF938C01C090BB02D090BC02E090BD02E4
:10339000F090BE028091B7029091B802A091B9025C
:1033A000B091BA02C82AD92AEA2AFB2ACFE1D0E092
:1033B000D701C6010C2E04C0B695A79597958795A1
:1033C0000A94D2F780FF06C0B8018C2F0E94E70450
:1033D000019721F4219760F780E001C08C2FDF91E5
:1033E000CF911F910F91FF90EF90DF90CF900895B4
:1033F000CF93DF93EC010E94B919BE010E94E7044C
:10340000DF91CF910895CB010E94F8190895809122
:10341000BF0285958595859508958091BF02877037
:10342000089598E0899F90011124262B2093BF02D4
:103430000C94FD182091BF02809582238093BF02D7
:10344000982F977069F430E0482F552747FD509525
:103450002417350729F08595859585950C941E19B7
:1034600008959091BF02977081E009F480E008957B
:1034700020910C0130910D01F90132969FEF40E04F
:103480005191581789F09F3F19F4511101C0942FA1
:103490004F5F4630A9F79F3F39F0F901E90FF11D61
:1034A00097FDFA9582830895089520910C0130913B
:1034B0000D01F9013296285F3F4F9081981301C0AA
:1034C00010823196E217F307C1F7089581E090E08A
:1034D000E0910C01F0910D01E80FF91F10820196A7
:1034E00088309105A9F708959091CB02892B80939C
:1034F000CB02089580959091CB0289238093CB02D3
:1035000008951092CB0208959091CA02892B80935E
:10351000CA02089580959091CA0289238093CA02B5
:1035200008951092CA0208959091C902892B809340
:10353000C902089580959091C90289238093C90298
:1035400008951092C90208958093C00208951092C0
:10355000C002089580910C0190910D01FC013196FB
:103560009C01285F3F4F80E0919191118F5FE2179E
:10357000F307D1F70895E0910C01F0910D018091CE
:10358000CB028083E0910C01F0910D01908180913C
:10359000CA02892B8083E0910C01F0910D0190818A
:1035A0008091C902892B80838091C002882361F0B9
:1035B000E0910C01F0910D019081892B80830E9494
:1035C000AA1A81111092C00280910C0190910D01F4
:1035D0000C94EA0F0E94C01480E00E9402030E9433
:1035E000AC210E94DE0F0C9419071F920F920FB6A8
:1035F0000F9211248F939F93AF93BF938091CD022D
:10360000811113C08091CE029091CF02A091D0027F
:10361000B091D1024196A11DB11D8093CE0290932D
:10362000CF02A093D002B093D102BF91AF919F91EE
:103630008F910F900FBE0F901F90189582E084BD60
:1036400093E095BD9AEF97BD80936E0008952FB7D4
:10365000F8948091CE029091CF02A091D002B091C7
:10366000D1022FBF0895CF92DF92EF92FF920F9376
:103670001F932FB7F8944091CE025091CF026091E2
:10368000D0027091D1022FBF6A017B01EE24FF248A
:103690008C0120E030E0C016D106E206F30610F4FB
:1036A000415051099A01281B390BC9011F910F91F3
:1036B000FF90EF90DF90CF9008951F920F920FB67A
:1036C0000F9211248F939F93AF93BF938091CE025B
:1036D0009091CF02A091D002B091D1020196A11D8C
:1036E000B11D8093CE029093CF02A093D002B093ED
:1036F000D102BF91AF919F918F910F900FBE0F900C
:103700001F9018950E949C0CF8942FEF87EA91E681
:10371000215080409040E1F700C0000087E090EB2E
:10372000DC018093ED029093EE02A093EF02B09340
:10373000F0029CE088E10FB6F894A89580936000B1
:103740000FBE90936000FFCFAF92BF92CF92DF92F7
:10375000EF92FF920F931F93CF93C3E0CC24C394B7
:10376000D12CE82EF12C8C2F0E94EF075C010CE08D
:1037700010E09601002E02C0220F331F0A94E2F7D8
:103780002A213B21232B51F0602F7C2F80E00E94C7
:103790008906E816F90611F481E006C00150110906
:1037A00040F7C15000F780E0CF911F910F91FF903B
:1037B000EF90DF90CF90BF90AF900895CF93C82F38
:1037C0008CE20E94A41B882321F08C2FCF910C94B3
:1037D000A41B80E0CF910895CF930E94341D8111E6
:1037E00002C00E94151DC5E6C15049F00E94740731
:1037F0008FE39CE90197F1F700C00000F5CF89E263
:103800000E94DE1B81110FC18AE20E94DE1B811122
:103810000E94151D85E00E94DE1B81110E94821B03
:103820000E943F1D8093CC0287E00E94DE1B88230C
:10383000A9F18BE10E94DE1B882351F08091CC021C
:1038400081FB222720F991E0922790FB81F90EC09D
:103850008EE00E94DE1B882361F08091CC0282FB07
:10386000222720F991E0922790FB82F98093CC02E5
:1038700015C080E10E94DE1B9091CC02882341F0AC
:1038800093FB222720F981E0822780FB93F904C073
:10389000892F809580FB90F99093CC028091CC0287
:1038A0000E94431D0E94511D90E09093DE02809380
:1038B000DD0280EE0E94DE1B882341F08091DD0254
:1038C000982F909590FB80F98093DD0289E30E9408
:1038D000DE1B882359F08091DD0281FB222720F92D
:1038E00091E0922790FB81F98093DD0282EE0E94A5
:1038F000DE1B882359F08091DD0282FB222720F90C
:1039000091E0922790FB82F98093DD0286EE0E947F
:10391000DE1B882359F08091DD0283FB222720F9EA
:1039200091E0922790FB83F98093DD0283EE0E9461
:10393000DE1B882359F08091DD0284FB222720F9C9
:1039400091E0922790FB84F98093DD0285E30E9449
:10395000DE1B882359F08091DD0285FB222720F9A8
:1039600091E0922790FB85F98093DD0281E30E942C
:10397000DE1B882359F08091DD0286FB222720F987
:1039800091E0922790FB86F98093DD0281E10E940D
:10399000DE1B882359F08091DD0287FB222720F966
:1039A00091E0922790FB87F98093DD028091DD0200
:1039B0000E94551D87E20E94DE1BC82F8EE10E94E7
:1039C000DE1B8111C2608FE10E94DE1B8111C46089
:1039D00080E20E94DE1B8111C86081E20E94DE1B32
:1039E0008111C06182E20E94DE1B8111C06283E20C
:1039F0000E94DE1B8111C06484E20E94DE1B8823CA
:103A000011F0C06802C0CC2329F08C2F0E944C1DFD
:103A10006C2F03C00E94481D682F70E080E090E08A
:103A2000CF910C948018CF9108956DEE7EEF80E0D9
:103A300090E00E94BF2360E082E090E00E94AD230E
:103A400060E083E090E00E94AD2360E084E090E0DD
:103A50000E94AD2360E085E090E00E94AD2360E02D
:103A600086E090E00C94AD2380E090E00E94A723D4
:103A700021E08D3E9E4F09F020E0822F089582E0E4
:103A800090E00C949F23682F82E090E00C94AD238B
:103A900083E090E00C949F23682F83E090E00C94E7
:103AA000AD2384E090E00C949F23682F84E090E0A5
:103AB0000C94AD2386E090E00C949F23682F86E061
:103AC00090E00C94AD238091D40280FF0BC06091F4
:103AD000110185E0689FB001112475956795759572
:103AE00067952BC081FF09C06091110185E0689F37
:103AF000B00111247595679520C082FF07C06091C1
:103B0000110185E0689FB001112417C09091D50282
:103B10009923D1F060911001961788F72091110137
:103B200085E0289F90011124929FA001939F500D42
:103B3000112470E0CA010E9471236038710540F4BD
:103B40006115710539F002C065E070E0862F0895B7
:103B50008FE7089581E008958091D40280FF08C026
:103B600060910F0170E0759567957595679521C017
:103B700081FF06C060910F0170E07595679519C0CF
:103B800082FF04C060910F0170E010C09091D502D7
:103B90009923C1F060910E019617A0F780910F0153
:103BA000899FC001112470E00E9471236038710563
:103BB00028F46115710521F0862F08958FE7089587
:103BC00081E0089561E070E0F4CF803F21F40E942D
:103BD000631D819504C0813F29F40E94631D809379
:103BE000D8020895823F21F40E94631D819504C08C
:103BF000833F29F40E94631D8093D7020895893F73
:103C000019F40E94AC1D05C08A3F31F40E94AC1D1E
:103C100081958093D90208958B3F21F40E94AC1DB9
:103C2000819504C08C3F29F40E94AC1D8093DA0278
:103C30000895843F21F48091D602816017C0853FAA
:103C400021F48091D602826011C0863F21F48091D8
:103C5000D60284600BC0873F21F48091D602886031
:103C600005C0883F31F48091D60280618093D602EE
:103C700008958D3F21F48091D40281600BC08E3F66
:103C800021F48091D402826005C08F3F29F4809195
:103C9000D40284608093D4020895803F39F48091E7
:103CA000D80287FF6CC01092D80269C0813F29F406
:103CB0008091D8021816BCF362C09091D702823F5F
:103CC00029F497FF5CC01092D70259C0833F19F4C2
:103CD0001916CCF354C0893F41F48091D9021816CB
:103CE0000CF04DC01092D9024AC08A3F29F480914D
:103CF000D90287FF44C0F6CF8B3F39F48091DA02B6
:103D000087FF3DC01092DA023AC08C3F29F48091BF
:103D1000DA021816BCF333C0843F21F48091D60236
:103D20008E7F17C0853F21F48091D6028D7F11C010
:103D3000863F21F48091D6028B7F0BC0873F21F410
:103D40008091D602877F05C0883F31F48091D602EA
:103D50008F7E8093D60213C08D3F21F48091D402D0
:103D60008E7F0BC08E3F21F48091D4028D7F05C0E1
:103D70008F3F29F48091D4028B7F8093D40280916D
:103D8000D70281110EC08091D80281110AC08091A2
:103D9000D902811106C08091DA02811102C010920D
:103DA000D502089586ED92E00E94F50F0E94271B30
:103DB0009093D3028093D20208951F93CF93DF9301
:103DC0008091D2029091D3020E94331BAC0190915A
:103DD000D502992321F02091120130E006C02091F4
:103DE00013018AE0289F900111244217530708F419
:103DF00086C08091D702C091D802D091D90210918B
:103E0000DA02811107C0C11176C0D11174C011113D
:103E100072C075C09F3F19F09F5F9093D50218162E
:103E200024F40E94631D8093D7028091D70287FFFC
:103E300005C00E94631D81958093D7021C1624F44F
:103E40000E94631D8093D8028091D80287FF05C02D
:103E50000E94631D81958093D8026091D7026623EA
:103E600039F1C091D802CC2319F1772767FD7095FD
:103E7000872F972F0E94762223E333E343E35FE308
:103E80000E94DA220E9443226093D7026C2F772788
:103E900067FD7095872F972F0E94762223E333E3E7
:103EA00043E35FE30E94DA220E9443226093D80238
:103EB0001D1624F40E94AC1D8093D9028091D90272
:103EC00087FF05C00E94AC1D81958093D902111611
:103ED00024F40E94AC1D8093DA028091DA0287FFFD
:103EE00005C00E94AC1D81958093DA02DF91CF91CD
:103EF0001F910C94D21E9F3F09F08ECF96CFDF9179
:103F0000CF911F910895E6EDF2E085E0DF011D926B
:103F10008A95E9F71092D5021092D4020895833061
:103F200081F128F4813059F08230D1F00895853044
:103F300009F449C0B8F1863009F456C0089580915B
:103F40001301262F30E0280F311D2F3F310524F4B7
:103F5000680F6093130108958FEF80931301089504
:103F600080911201262F30E0280F311D2F3F31059F
:103F700024F4680F6093120108958FEF809312016B
:103F8000089580911101262F30E0280F311D2F3F19
:103F9000310524F4680F6093110108958FEF809329
:103FA0001101089580911001262F30E0280F311D56
:103FB0002F3F310524F4680F6093100108958FEFAF
:103FC00080931001089580910F01262F30E0280F73
:103FD000311D2F3F310524F4680F60930F010895C0
:103FE0008FEF80930F01089580910E01262F30E00E
:103FF000280F311D2F3F310524F4680F60930E0107
:1040000008958FEF80930E010895833011F128F405
:10401000813049F0823091F00895853081F120F1AE
:104020008630C1F1089580911301681720F4861B32
:104030008093130108951092130108958091120145
:10404000681720F4861B80931201089510921201C4
:10405000089580911101681720F4861B8093110147
:10406000089510921101089580911001681720F4AD
:10407000861B80931001089510921001089580917D
:104080000F01681720F4861B80930F01089510928A
:104090000F01089580910E01681720F4861B80930C
:1040A0000E01089510920E0108950F931F93873209
:1040B00008F040C08E3108F08AC08E3009F474C018
:1040C000C0F4873009F45EC068F4863009F09AC005
:1040D0008091CC02817F8E7F8093CC0281E080939F
:1040E000DC0291C0883009F486C08B3009F483C0AB
:1040F00089C0863109F47FC068F4803109F082C03C
:104100008091CC0283FB222720F991E0922790FB3B
:1041100083F953C0893109F46EC08B3109F072C044
:104120008091CC0281FB222720F991E0922790FB1D
:1041300081F943C0883309F45EC050F4893209F430
:104140005CC0853309F459C0873209F456C05AC09F
:10415000833409F452C028F48A3308F453C08953D5
:1041600037C0883409F04EC00E94C0140FEF13ED21
:1041700020E3015010402040E1F700C000000E9401
:10418000821B39C09091CC02892F8095817080FB71
:1041900090F929F0966098609093CC0234C0997F92
:1041A000977F9093CC0227C08091CC0282FB22277C
:1041B00020F991E0922790FB82F98093CC02992319
:1041C000D1F08091CC0281608093CC0214C08D51DB
:1041D00041E050E060E070E08A019B0104C0000F04
:1041E000111F221F331F8A95D2F7C901B8010E94FF
:1041F00080180E94C01481E006C061E070E080E099
:1042000090E0F5CF80E01F910F91089580E0089530
:1042100080E008958E518A3030F4E82FF0E0E75CBA
:10422000FE4F8081089580E00895CF93C82F80913C
:10423000DC02813069F018F08230C9F183C0E0916E
:104240000C01F0910D018081823209F07DC007C020
:10425000E0910C01F0910D018081823261F48C2F8C
:104260000E940621811104C08C2F0E9455201DC080
:1042700081E090E01AC08C2F0E940821811114C0A7
:10428000C43179F048F4CB3079F0C03109F060C026
:1042900082E08093DC0208C0C93219F0C83321F0F3
:1042A00057C01092DC0254C081E0817053C0C93203
:1042B00089F118F5C43171F1B0F4C73009F046C086
:1042C0008EE18093130182E3809312018AE0809350
:1042D000110184E18093100188E080930F0188E24E
:1042E00080930E0133C082EE8C0F863078F58C2FD0
:1042F0000E940A218093DB0229C0CE34E9F020F429
:10430000CB3421F56AE013C0C13579F0C235F1F440
:1043100061E00DC08091DB02882319F01092DB026E
:1043200015C081E08093DC0215C061E006C0809179
:10433000DB020E948F1F0AC06AE08091DB020E94AC
:10434000052004C01092DC0280E004C081E002C0BD
:1043500080E0ABCFCF9108950E94341D811102C03F
:104360000E94151D0E945A1D8093EC0280FF02C01E
:10437000869501C080E00C9402038091EC02982F96
:104380009695292F30E0233031054CF49F5F990F2B
:104390008170892B81608093EC020E945E1D809168
:1043A000EC0286950C9402038091EC02982F96956E
:1043B00091F09158990F8170892B8093EC028E7F38
:1043C00091E009F490E08091EC0290FB80F98093F9
:1043D000EC020E945E1D8091EC0286950C94020313
:1043E0008091EC02982F909590FB80F98093EC02DD
:1043F0000E945E1D8091EC0280FF02C0869501C084
:1044000080E00C9402039091EC02892F86958F5FD7
:104410008F779170843028F4880F892B8093EC0279
:1044200002C09093EC028091EC028E7F91E009F43F
:1044300090E08091EC0290FB80F98093EC020E9466
:104440005E1D8091EC0286950C9402032091EC0293
:10445000922F96958927982F990F822F8170892BFB
:104460008093EC028E7F91E009F490E08091EC0261
:1044700090FB80F98093EC020E945E1D8091EC021B
:1044800086950C94020304D06894B1118DC00895F0
:1044900070D088F09F5790F0B92F9927B751A0F0AE
:1044A000D1F0660F771F881F991F1AF0BA95C9F7C8
:1044B00012C0B13081F077D0B1E0089574C0672F99
:1044C000782F8827B85F39F0B93FCCF38695779578
:1044D0006795B395D9F73EF4909580957095619561
:1044E0007F4F8F4F9F4F0895E89409C097FB3EF48C
:1044F00090958095709561957F4F8F4F9F4F992331
:10450000A9F0F92F96E9BB279395F69587957795AE
:104510006795B795F111F8CFFAF4BB0F11F460FF6E
:104520001BC06F5F7F4F8F4F9F4F16C0882311F0C6
:1045300096E911C0772321F09EE8872F762F05C0DA
:10454000662371F096E8862F70E060E02AF09A9575
:10455000660F771F881FDAF7880F9695879597F96A
:10456000089557FD9058440F551F59F05F3F71F063
:104570004795880F97FB991F61F09F3F79F08795CA
:104580000895121613061406551FF2CF4695F1DF53
:1045900008C0161617061806991FF1CF86957105E3
:1045A000610508940895E894BB2766277727CB0117
:1045B00097F908950BD078C069D028F06ED018F024
:1045C000952309F05AC05FC01124EECFCADFA0F3D3
:1045D000959FD1F3950F50E0551F629FF001729F98
:1045E000BB27F00DB11D639FAA27F00DB11DAA1FB7
:1045F000649F6627B00DA11D661F829F2227B00D04
:10460000A11D621F739FB00DA11D621F839FA00D8E
:10461000611D221F749F3327A00D611D231F849FDE
:10462000600D211D822F762F6A2F11249F57504035
:104630008AF0E1F088234AF0EE0FFF1FBB1F661FD0
:10464000771F881F91505040A9F79E3F510570F089
:1046500014C0AACF5F3FECF3983EDCF386957795C4
:104660006795B795F795E7959F5FC1F7FE2B880F84
:10467000911D9695879597F9089597F99F6780E81A
:1046800070E060E008959FEF80EC089500240A94A4
:104690001616170618060906089500240A9412161D
:1046A0001306140605060895092E0394000C11F450
:1046B000882352F0BB0F40F4BF2B11F460FF04C0FD
:1046C0006F5F7F4F8F4F9F4F0895991B79E004C014
:1046D000991F961708F0961B881F7A95C9F7809541
:1046E000089597FB072E16F4009407D077FD09D0A4
:1046F0000E948B2307FC05D03EF4909581959F4F37
:104700000895709561957F4F0895EE0FFF1F0590F6
:10471000F491E02D0994AA1BBB1B51E107C0AA1F0D
:10472000BB1FA617B70710F0A61BB70B881F991F52
:104730005A95A9F780959095BC01CD010895F999F6
:10474000FECF92BD81BDF89A992780B50895A8E162
:10475000B0E042E050E00C94C723262FF999FECF39
:1047600092BD81BDF89A019700B4021639F01FBAC4
:1047700020BD0FB6F894FA9AF99A0FBE08950196E3
:10478000272F0E94AE230C94AD23DC01CB01FC014A
:10479000F999FECF06C0F2BDE1BDF89A319600B49A
:0E47A0000D9241505040B8F70895F894FFCFA5
:1047AE00FFF9072309DF08AB08FC0701C10228083F
:1047BE00140A321E4F7953636676496959091929CD
:1047CE00030F1F5F43404D36201405C7049104713B
:1047DE0004FD0316042F0448040102030405060712
:0447EE0008090000B6
:00000001FF
